:100000000C9473030C9490030C9490030C94900341
:100010000C9490030C9490030C9490030C94900314
:100020000C9490030C9490030C9490030C94900304
:100030000C9490030C9490030C9475080C9490030A
:100040000C9490030C941C050C94BF040C94810434
:100050000C9490030C94B2150C9490030C949003A0
:100060000C9490030C949003426175647261746502
:10007000206F666620627920256C646270730A00C6
:10008000756E6974203C205345525F434E540062A4
:100090006572746F732F6370752F6176722F64723F
:1000A000762F7365725F6D6567612E630073697A81
:1000B00065203E203100626572746F732F73747215
:1000C0007563742F6669666F6275662E6800666474
:1000D0002D3E68772D3E72786275666665720062A5
:1000E0006572746F732F6472762F7365722E63005E
:1000F00066642D3E68772D3E74786275666665721B
:1001000000626572746F732F6472762F7365722E3E
:1001100063002166642D3E69735F6F70656E0062D7
:100120006572746F732F6472762F7365722E63001D
:10013000756E6974203C20636F756E746F662873EA
:1001400065725F68616E646C6573290062657274C4
:100150006F732F6472762F7365722E6300706F72E7
:10016000742D3E69735F6F70656E00626572746FA7
:10017000732F6472762F7365722E630066642D3E52
:100180005F74797065203D3D204B46545F53455266
:1001900049414C00626572746F732F6472762F73DD
:1001A00065722E68002174696D65725F696E69748D
:1001B00069616C697A656400626572746F732F643B
:1001C00072762F74696D65722E63002674696D6591
:1001D000722D3E6C696E6B00626572746F732F6472
:1001E00072762F74696D65722E630066642D3E729F
:1001F00065616400626572746F732F696F2F6B663F
:10020000696C652E680066642D3E777269746500BE
:10021000626572746F732F696F2F6B66696C652EE0
:1002200068006275665F706F696E746572203E3D2E
:100230002062756600626572746F732F6D776172EC
:10024000652F666F726D617477722E6300636861EB
:100250006E6E656C00626572746F732F6E65742FBD
:10026000617832352E630063747800626572746F52
:10027000732F6E65742F617832352E630069736158
:100280006C6E756D286329207C7C2063203D3D20A9
:1002900027202700626572746F732F6E65742F615B
:1002A0007832352E63006374782D3E6372635F6F1E
:1002B0007574203D3D20415832355F4352435F43C2
:1002C0004F525245435400626572746F732F6E65CE
:1002D000742F617832352E6300706174685F6C65CD
:1002E0006E203E3D203200626572746F732F6E6522
:1002F000742F617832352E63007061746800626516
:1003000072746F732F6E65742F617832352E6300AF
:1003100066642D3E636C656172657272006265721F
:10032000746F732F696F2F6B66696C652E6800663A
:10033000642D3E6572726F7200626572746F732F06
:10034000696F2F6B66696C652E680025733A204FC4
:100350006E6C79206672616D657320776974686F61
:100360007574206C61796572332070726F746F637D
:100370006F6C206172652068616E646C65642C200E
:10038000676F74205B253032585D0A0025733A2070
:100390004F6E6C79205549206672616D65732061DE
:1003A00072652068616E646C65642C20676F7420D0
:1003B0005B253032585D0A0025733A204368616E30
:1003C0006E656C206572726F72205B253034785DCB
:1003D0000A000000891112239B322446AD5736656E
:1003E000BF74488CC19D5AAFD3BE6CCAE5DB7EE9B1
:1003F000F7F88110080193331A22A5562C47B775D8
:100400003E64C99C408DDBBF52AEEDDA64CBFFF990
:1004100076E802218B30100299132667AF763444B8
:10042000BD554AADC3BC588ED19F6EEBE7FA7CC870
:10043000F5D983310A2091121803A7772E66B55497
:100440003C45CBBD42ACD99E508FEFFB66EAFDD850
:1004500074C904428D5316619F702004A915322778
:10046000BB364CCEC5DF5EEDD7FC6888E1997AAB30
:10047000F3BA85520C4397711E60A1142805B33757
:100480003A26CDDE44CFDFFD56ECE9986089FBBB10
:1004900072AA06638F7214409D512225AB34300638
:1004A000B9174EEFC7FE5CCCD5DD6AA9E3B8788AF0
:1004B000F19B87730E6295501C41A3352A24B11617
:1004C0003807CFFF46EEDDDC54CDEBB962A8F99AD0
:1004D000708B088481951AA793B62CC2A5D33EE1F0
:1004E000B7F04008C919522BDB3A644EED5F766DC8
:1004F000FF7C899400859BB712A6ADD224C3BFF1BF
:1005000036E0C1184809D33B5A2AE55E6C4FF77DA7
:100510007E6C0AA583B4188691972EE3A7F23CC09F
:10052000B5D14229CB38500AD91B666FEF7E744C87
:10053000FD5D8BB502A499961087AFF326E2BDD07E
:1005400034C1C3394A28D11A580BE77F6E6EF55C67
:100550007C4D0CC685D71EE597F42880A1913AA35F
:10056000B3B2444ACD5B5669DF78600CE91D722F47
:10057000FB3E8DD604C79FF516E4A9902081BBB33E
:1005800032A2C55A4C4BD7795E68E11C680DF33F27
:100590007A2E0EE787F61CC495D52AA1A3B038821F
:1005A000B193466BCF7A5448DD59622DEB3C700E07
:1005B000F91F8FF706E69DD414C5ABB122A0B992FE
:1005C0003083C77B4E6AD5585C49E33D6A2CF11EE7
:1005D000780F6368203C3D2035004D6F64656D2FBA
:1005E00068617264776172652E630066642D3E5F98
:1005F00074797065203D3D204B46545F4146534B16
:10060000004D6F64656D2F6166736B2E680080818D
:1006100083848687898A8C8E8F9192949597989AF5
:100620009B9D9EA0A2A3A5A6A7A9AAACADAFB0B260
:10063000B3B5B6B7B9BABCBDBEC0C1C2C4C5C6C8E1
:10064000C9CACBCDCECFD0D2D3D4D5D6D7D9DADB89
:10065000DCDDDEDFE0E1E2E3E4E5E6E7E8E9EAEA63
:10066000EBECEDEEEEEFF0F1F1F2F3F3F4F5F5F67D
:10067000F6F7F8F8F9F9FAFAFAFBFBFCFCFCFDFDD9
:10068000FDFDFEFEFEFEFEFFFFFFFFFFFFFF6275AA
:10069000665F706F696E746572203E3D206275669C
:1006A00000626572746F732F6D776172652F666F6C
:1006B000726D617477722E6300203D203078257052
:1006C0000A00496E76616C6964207074723A200089
:1006D0003A2000417373657274696F6E20666169B8
:1006E0006C65643A200011241FBECFEFD8E0DEBF56
:1006F000CDBF11E0A0E0B1E0ECE8F1E502C005906B
:100700000D92AE3DB107D9F716E0AEEDB1E001C0F4
:100710001D92A232B107E1F70E94DE140C94C428A6
:100720000C9400001092C00088E98093C1000895E5
:100730001092C1000895FC012285211105C021E01D
:10074000228788EB8093C1000895E2ECF0E080817D
:1007500094E0660F771F9A95E1F78F7C862B808354
:1007600008959FB7F89484B1886284B99FBF8FB70A
:10077000F894229A8FBF8FB7F89424988FBF80ED9A
:100780008CBD8CB581608CBD8DB58E7F8DBD08957F
:100790001CBC9FB7F89484B1837C84B99FBF089533
:1007A00008950895FC01828508956FB7F894DC01DF
:1007B0001A962C911A97211120C0E091E105F09131
:1007C000E205478D50A121A132A142175307A9F09C
:1007D00021E01A962C93A78DB0A185A196A1A81708
:1007E000B90719F483A194A104C0A78DB0A1CD01CC
:1007F000019690A3878F8C918EBD6FBF08954F9205
:100800005F926F927F928F929F92AF92BF92CF92A0
:10081000DF92EF92FF92CF93DF934A015B01CB010E
:10082000BA019695879577956795605C7D4B804F6B
:100830009F4FA50194010E946C28E901219744274C
:10084000552760E472E48FE090E00E94342875013F
:100850006401C61AD70AE80AF90A26013701F7FE29
:1008600007C04424552432014C185D086E087F08E7
:10087000C501B40121E230E040E050E00E946C2864
:10088000241535054605570580F4FF92EF92DF9257
:10089000CF9288E690E09F938F930E945C250F9003
:1008A0000F900F900F900F900F90D093C500C093B2
:1008B000C400DF91CF91FF90EF90DF90CF90BF9079
:1008C000AF909F908F907F906F905F904F90089522
:1008D000CF93DF93EC018230910544F04AE953E075
:1008E0006FE870E080E890E00E94DE252BE02C9F0E
:1008F000C0012D9F900D11248A5F9E4FDF91CF91F3
:1009000008951F920F920FB60F9211242F933F93C9
:100910008F939F93AF93BF93EF93FF93E091DF0586
:10092000F091E005278D30A181A192A12817390708
:1009300031F488E98093C1001092100113C0A78D93
:10094000B0A185A196A1A817B90719F483A194A114
:1009500004C0A78DB0A1CD01019690A3878F8C9183
:100960008093C600FF91EF91BF91AF919F918F91BE
:100970003F912F910F900FBE0F901F9018951F92CF
:100980000F920FB60F9211242F933F934F935F93C3
:100990008F939F93AF93BF93EF93FF93E091DF0506
:1009A000F091E00597A58091C0008871892B87A7F9
:1009B0005091C60027A130A583A594A52817390713
:1009C00039F421A532A585A596A52817390761F028
:1009D00021A532A587A190A5019741E028173907E5
:1009E00009F040E0842F01C081E080FF04C087A5AA
:1009F000816087A712C0A1A5B2A55C9321A532A5ED
:100A000085A596A52817390719F483A594A503C0D1
:100A100081A592A5019692A781A7FF91EF91BF9121
:100A2000AF919F918F915F914F913F912F910F9037
:100A30000FBE0F901F9018951F920F920FB60F9236
:100A400011242F933F934F938F939F93AF93BF9313
:100A5000EF93FF93E091E105F091E20527A130A526
:100A600083A594A52817390739F421A532A585A5B2
:100A700096A52817390761F021A532A587A190A571
:100A8000019741E02817390709F040E0842F01C0A1
:100A900081E080FD13C08EB5A1A5B2A58C9321A5E0
:100AA00032A585A596A52817390719F483A594A51D
:100AB00003C081A592A5019692A781A7E091E105C7
:100AC000F091E205278D30A181A192A12817390765
:100AD00099F0A78DB0A185A196A1A817B90719F41F
:100AE00083A194A104C0A78DB0A1CD01019690A3CC
:100AF000878F8C918EBD02C010921B01FF91EF91E8
:100B0000BF91AF919F918F914F913F912F910F90F6
:100B10000FBE0F901F9018959FB7F89483E085BB88
:100B200014BC15BC82E084BD85B5836085BD16BC50
:100B300089EF87BDEEE6F0E080818E7F8083808143
:100B4000826080839FBF0895CF93DF93EC01FB0108
:100B50005FB7F894278D30A183A194A12817390796
:100B6000E9F421A132A185A196A128173907B1F492
:100B700081E05FBF80FD11C04FB7F894A1A1B2A181
:100B8000CC9321A132A185A196A12817390799F408
:100B900083A194A192A381A314C0DACF81A192A1D1
:100BA000278D30A12150310941E08217930709F0C8
:100BB00040E0842FDECF21A132A12F5F3F4F32A32F
:100BC00021A34FBF80A991A9DC01ED91FC91008484
:100BD000F185E02D0995CE019927DF91CF910895F8
:100BE000FC014FB7F89427A130A581A592A54FBF6E
:100BF0002817390739F087A5897B79F024C087A5A4
:100C0000897BC9F74FB7F89427A130A581A592A594
:100C10004FBF2817390799F3EECF2FB7F894A7A144
:100C2000B0A585A596A5A817B90719F483A594A51D
:100C300004C0A7A1B0A5CD01019690A787A38C9170
:100C40002FBF90E008958FEF9FEF0895AF92BF926E
:100C5000CF92DF92EF92FF920F931F93CF93DF9388
:100C60007C015B016A01FC010089118922893389B9
:100C70000C3412452544334541F04CEB50E064E917
:100C800071E08CE791E00E94DE25E50100E010E0D4
:100C90000C151D0559F0C7010E94F0058F3F2FEF7D
:100CA000920721F00F5F1F4F8993F2CFC801DF91A8
:100CB000CF911F910F91FF90EF90DF90CF90BF9059
:100CC000AF900895AF92BF92CF92DF92EF92FF92D2
:100CD0000F931F93CF93DF937C015B016A01FC01AB
:100CE00000891189228933890C3412452544334502
:100CF00041F04CEB50E064E971E08CE791E00E9438
:100D0000DE25E50100E010E00C151D0561F089917C
:100D1000B701992787FD90950E94A405019619F0C7
:100D20000F5F1F4FF1CFC801DF91CF911F910F913E
:100D3000FF90EF90DF90CF90BF90AF900895CF934A
:100D4000DF93EC01488959896A897B894C34524583
:100D50006544734541F04CEB50E064E971E08CE789
:100D600091E00E94DE258FA590E0DF91CF9108955C
:100D7000CF93DF93EC01488959896A897B894C3488
:100D800052456544734541F04CEB50E064E971E035
:100D90008CE791E00E94DE251FA6DF91CF91089598
:100DA000CF93DF93EC01488959896A897B894C3458
:100DB00052456544734549F04CEB50E064E971E0FD
:100DC0008CE791E00E94DE2500C02F8D38A189A11B
:100DD0009AA128173907C9F788A999A9DC01ED91CB
:100DE000FC910284F385E02D09958111EECF80E01E
:100DF00090E0DF91CF910895EF92FF920F931F93B0
:100E0000CF93DF93EC018B016230710540F042E635
:100E100051E06CE471E080E391E00E94DE25F8018E
:100E2000EE0FFF1FE152FA4FD183C0838E8D8823CE
:100E300041F045E651E06FE171E082E191E00E940E
:100E4000DE2581E08E8F1D8F0C8FC8010E94680403
:100E500099AB88ABDC0112968D919C911397892BED
:100E600041F44DE651E061E071E080EF90E00E94D6
:100E7000DE25E8A9F9A984819581892B41F44EE604
:100E800051E06FED70E08EEC90E00E94DE25E8A965
:100E9000F9A9E680F78002811381B2E0EB16F10434
:100EA00040F441E251E066EB70E08DEA90E00E9490
:100EB000DE251CA30BA31AA309A318A30F8FC70138
:100EC0000197800F911F9EA38DA3E8A9F9A9E08443
:100ED000F18404811581E2E0EE16F10440F441E270
:100EE00051E066EB70E08DEA90E00E94DE251CA7E1
:100EF0000BA71AA709A718A70FA3C7010197800F6F
:100F0000911F9EA78DA788A999A9DC01ED91FC915D
:100F10000190F081E02DBE0109951FA6CE01DF9161
:100F2000CF911F910F91FF90EF900895FC014FB763
:100F3000F89427A130A581A592A54FBF281739079E
:100F4000B1F02FB7F894A7A1B0A585A596A5A817CD
:100F5000B90719F483A594A504C0A7A1B0A5CD0134
:100F6000019690A787A38C912FBF90E008958FEFF3
:100F70009FEF08956FB7F894FC0147A150A521A5F4
:100F800032A56FBF81E04217530709F480E008954E
:100F9000DC01D0968D919C91D197DC01ED91FC9173
:100FA0000480F581E02D09944FB7F894FC0121A548
:100FB00032A530A727A34FBF08954FB7F894FC017F
:100FC00021A132A130A3278F4FBF0895CF93DF9384
:100FD000EC010E94D407CE01DF91CF910C94DD0784
:100FE000CF93DF93EC01488959896A897B894C3416
:100FF00052456544734541F04CEB50E064E971E0C3
:101000008CE791E00E94DE258E8D811108C04BE8AF
:1010100051E06BE671E08DE591E00E94DE251E8EC9
:10102000CE010E94D00688A999A9DC01ED91FC911E
:101030000280F381E02D099519AA18AACE010E9419
:10104000E60780E090E0DF91CF910895CF93DF93A2
:10105000EC01488959896A897B894C345245654439
:10106000734541F04CEB50E064E971E08CE791E0AE
:101070000E94DE25CE010E94F0076C8D7D8DCE0191
:101080000E94FC06CE01DF91CF910895FC01CB01B7
:1010900022E3DF011D922A95E9F74CE452E565E46D
:1010A00073E5408B518B628B738B26E238E035837E
:1010B000248320EF37E03783268326E236E031832E
:1010C000208322E636E03383228320ED36E0338727
:1010D00022872FE936E03587248728EB36E03787EB
:1010E0002687BC01CF010C94FC061F920F920FB60D
:1010F0000F9211240F931F932F933F934F935F935E
:101100006F937F938F939F93AF93BF93CF93DF930F
:10111000EF93FF938091E3059091E405A091E5059D
:10112000B091E6050196A11DB11D8093E305909352
:10113000E405A093E505B093E6050BEA1AEBC09130
:101140001E02D0911F0288819981892BD1F18FB71E
:10115000F8944091E3055091E4056091E5057091A4
:10116000E6058FBF88859985AA85BB85481B590BE5
:101170006A0B7B0B77FD25C0CF3FD10509F048F402
:101180002BEC30E048ED51E06BEC71E0CE010E94B9
:10119000F425EA81FB818881998191838083E881AC
:1011A000F9818A819B81938382831B821A821982AF
:1011B00018821B8B0A8BEC85FD85CE010C96099558
:1011C000BECFFF91EF91DF91CF91BF91AF919F91F2
:1011D0008F917F916F915F914F913F912F911F91CF
:1011E0000F910F900FBE0F901F90189582E292E022
:1011F00090931F0280931E021092210210922002EF
:1012000010922302109222028EE192E09093250226
:10121000809324021092E3051092E4051092E505F4
:101220001092E6050E948C058091E705882341F025
:1012300041E951E068EB71E085EA91E00E94DE252A
:1012400081E08093E7050895EF92FF920F931F933B
:10125000CF93DF931F92CDB7DEB77C018B018983DB
:10126000DB0112968D919C911397892B41F44EE0EE
:1012700051E060E172E086E092E00E94DE25D80154
:101280001296ED91FC91139741E050E0BE016F5F23
:101290007F4FC8010995019719F4C701992702C02A
:1012A0008FEF9FEF0F90DF91CF911F910F91FF90E4
:1012B000EF9008950F931F93CF93DF931F92CDB7B5
:1012C000DEB78C01DC018D919C91892B41F442EFBA
:1012D00050E064EF71E08BEE91E00E94DE25D801D2
:1012E000ED91FC9141E050E0BE016F5F7F4FC8017E
:1012F0000995019719F4898190E002C08FEF9FEF63
:101300000F90DF91CF911F910F910895CF93DF93AD
:10131000CDB7DEB79E01275F3F4F4D815E8164E20E
:1013200079E08F8198850E94B309DF91CF9108956C
:101330000F931F93CF93DF938C01EB018991882347
:1013400059F0B801992787FD90950E9424098F3F95
:101350002FEF920799F702C080E090E0DF91CF91E4
:101360001F910F9108952F923F924F925F926F922B
:101370007F928F929F92AF92BF92CF92DF92EF9225
:10138000FF920F931F93CF93DF93CDB7DEB7C45A6D
:10139000D1090FB6F894DEBF0FBECDBFFC01C85611
:1013A000DF4F79836883C859D040C656DF4F5983D1
:1013B0004883CA59D0405901C257DF4F1982188259
:1013C000CE58D0409E012F5F3F4FC957DF4F398322
:1013D0002883C758D040AE014A575F4FC757DF4FE9
:1013E00059834883C958D0409F012F5F3F4FC4564F
:1013F000DF4F39832883CC59D0408081853291F1E9
:10140000882309F427C7C656DF4F68817981CA59F6
:10141000D040C856DF4FE881F981C859D0400995BE
:10142000C257DF4FC880D980CE58D040FFEFCF1AC7
:10143000DF0AC557DF4FB982A882CB58D040C257C8
:10144000DF4FD982C882CE58D040C557DF4FA88021
:10145000B980CB58D040C456DF4FE881F981CC59D0
:10146000D040C2CF8181853251F4AF014E5F5F4FD2
:10147000C456DF4F59834883CC59D040C4CFC4569B
:10148000DF4FA881B981CC59D040C256DF4F1882B6
:10149000CE59D040C357DF4F1882CD58D040CF56D9
:1014A000DF4F1882C159D040CE56DF4F1882C25943
:1014B000D040FD018D918B3209F45EC060F4803222
:1014C000E9F0833209F05FC031E0C357DF4F388362
:1014D000CD58D040EECF8D3251F0803309F053C05B
:1014E00041E0C256DF4F4883CE59D040E2CF21E0E1
:1014F000CF56DF4F2883C159D040DBCF392D3C7FF9
:10150000932ECE56DF4F4881C259D040942ACD56F3
:10151000DF4F5881C359D04050FB92F8CF56DF4F70
:101520008881C159D04080FB93F8C057DF4F988124
:10153000C059D04090FB94F8CC56DF4FE881C45995
:10154000D040E0FB95F8C357DF4FF881CD58D0402D
:10155000F0FB96F8CB56DF4F2881C559D04020FBD1
:1015600097F8892D837009F0A4CF81E0CE56DF4F24
:101570008883C259D0409DCF51E0CE56DF4F58836B
:10158000C259D04096CFC357DF4F9881CD58D04035
:10159000C056DF4F9883C05AD0408A3229F0DF010D
:1015A000212C312C2AE013C0C5010296D5012D90C3
:1015B0003C9037FE09C0319421943108B1E0CF56F8
:1015C000DF4FB883C159D04031965C0112C0FD0194
:1015D0008D9190ED980F9A3060F4F1012E9F1001DB
:1015E0002F9F300C1124F0E32F1A3108280E311CE4
:1015F000EECFCF56DF4F2881C159D040222329F0AA
:10160000C256DF4F1882CE59D04080818E3221F5EC
:1016100081818A3231F0DF011196612C712C2AE030
:1016200009C0D5016D907C90329695012E5F3F4F99
:10163000590115C0FD018D9190ED980F9A3078F405
:10164000A301249F3001259F700C112450E3651ADB
:101650007108680E711CEECF66246A94762CDF0147
:101660008D918836D9F018F48C3459F01FC08C361F
:1016700041F08A37D9F4C057DF4F1882C059D040A3
:1016800006C081E0C057DF4F8883C059D040FD01BC
:10169000CC56DF4F1882C459D04012C0FD0191E0F2
:1016A000CC56DF4F9883C459D04005C0CC56DF4F8D
:1016B0001882C459D040C057DF4F1882C059D0405B
:1016C000DF011196C456DF4FB983A883CC59D040AF
:1016D0008080B5E68B1609F408C2B815ECF023E556
:1016E000821609F453C0281564F035E4831609F412
:1016F000FCC147E4841609F4F0C1882009F465C4EC
:101700002AC053E6851671F158150CF4CBC088E554
:10171000881609F48DC01FC090E7891609F471C0BE
:10172000981564F0A7E68A1609F4D7C18A160CF456
:10173000DBC1B9E68B1609F4B5C00DC0E5E78E161E
:1017400009F476C0F8E78F1609F46DC023E782121A
:1017500002C0D12C1DC0C557DF4FB982A882CB581B
:10176000D0403FC4A5014E5F5F4FC557DF4F59833F
:101770004883CB58D040D5018C918983D12C8E01E0
:101780000E5F1F4FFE0131965F0139C4DD24D394F3
:1017900095012E5F3F4FC557DF4F39832883CB58C4
:1017A000D040D501AD90BC90A114B10421F4A0E2C9
:1017B000AA2EA1E0BA2E77FE04C0F0E16F2EF7E268
:1017C0007F2E8501DD20C1F0F8018491882309F482
:1017D00016C4C8018A199B09861597050CF00FC419
:1017E0000F5F1F4FF1CFC8018A199B098615970516
:1017F0000CF005C40F5F1F4FD8018C918111F3CFFE
:10180000FEC3F5013296C557DF4FF983E883CB5805
:10181000D040D5016D917C9180E090E0EBE6EE2E1A
:10182000E1E0FE2E2BC07BE7E72E71E0F72E04C02F
:101830006BE6E62E61E0F62EC057DF4FB881C05947
:10184000D040BB2371F0F5013496C557DF4FF983C3
:10185000E883CB58D040D5016D917D918D919C91BD
:101860000DC0C5010296F50160817181C557DF4F3A
:1018700099838883CB58D04080E090E021E0CD561A
:10188000DF4F2883C359D04035E7831205C0CD56BA
:10189000DF4F1882C359D040CE56DF4F1882C2594D
:1018A000D04042C0C057DF4F4881C059D040442388
:1018B00071F0C5010496C557DF4F99838883CB58D3
:1018C000D040D5016D917D918D919C910FC0F50116
:1018D0003296C557DF4FF983E883CB58D040D50106
:1018E0006D917C91882777FD8095982F97FF13C085
:1018F00090958095709561957F4F8F4F9F4FCD56F6
:10190000DF4F1882C359D040B2E0CE56DF4FB883C4
:10191000C259D04005C0CD56DF4F1882C359D040C0
:101920005BE6E52E51E0F52EE1E0CB56DF4FE88394
:10193000C559D040611571058105910529F4CB5633
:10194000DF4F1882C559D0406114710441F4CB5661
:10195000DF4FF881C559D040FF2309F47CC0CD5634
:10196000DF4F2881C359D0408E010A571F4F2130C5
:10197000A9F02AE030E040E050E00E946C28F70136
:10198000E60FF71F8081D8018E938D01B901CA013E
:10199000611571058105910561F715C0FB01EF70B7
:1019A000FF27EE0DFF1D2081F80122938F0144E0F7
:1019B00096958795779567954A95D1F76115710545
:1019C0008105910559F777FE49C0C256DF4FF8816E
:1019D000CE59D040FF2309F441C0292D2C7F922EEF
:1019E000CE56DF4F3881C259D040932ACD56DF4FB3
:1019F0004881C359D04040FB92F8CF56DF4F588101
:101A0000C159D04050FB93F8C057DF4F8881C0596F
:101A1000D04080FB94F8CC56DF4F9881C459D04019
:101A200090FB95F8C357DF4FA881CD58D040A0FB5D
:101A300096F8CB56DF4FB881C559D040B0FB97F828
:101A4000292D237081E090E011F480E090E03101D5
:101A5000681A790A03C08E010A571F4FC757DF4F14
:101A600088819981C958D040801B910BF80120E3EF
:101A70005F01861597051CF422930196F9CFC35791
:101A8000DF4FE881CD58D040EE23A1F0CB56DF4F99
:101A9000F881C559D040FF2369F0882D8F7D8835A6
:101AA00049F4F5013197808222E0A21AB10880E35F
:101AB000D5018C93C957DF4FE881F981C758D040D1
:101AC000AE16BF0608F095C247EB52E065E372E040
:101AD00082E292E00E94DE258CC28A948A9411E010
:101AE0006114710449F002C0812C10E077FE07C038
:101AF00026E0622E712C03C066246394712C95013C
:101B00002C5F3F4FC557DF4F39832883CB58D040D8
:101B1000D501CD90DD90ED90FC9020E030E0A90162
:101B2000C701B6010E947E2687FF0AC0F7FAF0942B
:101B3000F7F8F094B2E0CE56DF4FB883C259D040E8
:101B4000C156DF4F1883CF59D040AA24A394B12C9B
:101B5000AC0EBD1EA20CB31C20E030E040E85FE3F9
:101B6000C701B6010E94CD2787FD32C0412C512C00
:101B700027EB33E44AEB51E5C701B6010E94CD27BC
:101B800087FD0EC029EF32E045E150E5C701B601FF
:101B90000E9482266B017C01EAE04E0E511CE8CFC8
:101BA00020E030E040E251E4C701B6010E94CD27B9
:101BB00087FD49C020E030E040E251E4C701B601B2
:101BC0000E9482266B017C01FFEF4F1A5F0AE8CF6B
:101BD00020E030E0A901C701B6010E947E26412C19
:101BE000512C882381F12FEF36EE4BED5EE2C701D9
:101BF000B6010E947E26181674F029EF32E045E106
:101C000050E5C701B6010E94D1276B017C012AE093
:101C1000421A5108E8CF20E030E040E85FE3C70116
:101C2000B6010E947E2687FF0EC020E030E040E231
:101C300051E4C701B6010E94D1276B017C0131E05C
:101C4000431A5108E8CF112301F14614570444F414
:101C50004CEF44164FEF54061CF064187508812CA5
:101C600051E0651A710881E0C357DF4F9881CD5864
:101C7000D0409827C156DF4F9883CF59D040A1E07C
:101C8000C357DF4FA883CD58D04081104BC057FEBB
:101C90003DC080E3E1E0F0E0EC0FFD1FE20DF31D3D
:101CA0008083F5016114710459F4C357DF4FB88183
:101CB000CD58D040B11104C0319680E090E006C00C
:101CC00032968EE2D50111968C93C30192012F5F5B
:101CD0003F4F280F391F40E38F018217930729F0E8
:101CE000009719F041930197F7CF93012095309514
:101CF000421653060CF4D1C03C01E1E0F0E0CA56B4
:101D0000DF4FF983E883C659D0405CC022273327D0
:101D100024193509CA56DF4F39832883C659D04064
:101D2000850150C08501CA56DF4F19821882C659F5
:101D3000D04048C0C701B6010E94EA26CF55DF4F08
:101D4000688379838A839B83C15AD040CF55DF4F04
:101D500048815981C15AD040BA01882777FD8095C2
:101D6000982F0E941D279B01AC01C701B6010E945C
:101D7000192620E030E040E251E40E94D1276B01B7
:101D80007C0198012F5F3F4FCF55DF4F8881C15AAB
:101D9000D040805DD8018C93CA56DF4F88819981ED
:101DA000C659D0400196CA56DF4FE881F981C6591D
:101DB000D040EF2B91F0CA56DF4F99838883C659E4
:101DC000D0408901CA56DF4F28813981C659D04099
:101DD000621673060CF0AECF14C06114710439F4AE
:101DE000C357DF4FF881CD58D040FF2339F0980119
:101DF0002E5F3F4FEEE2D8011196EC9381E090E028
:101E0000DACF20E030E040EA50E4C701B6010E949A
:101E1000CD2787FD42C0F80181E090E030E32291B8
:101E20002E3251F0820F8A3321F0808380E090E0DF
:101E300003C0308381E090E0AE16BF0680F3892BAB
:101E400061F18820B9F0F801AE16BF0678F4DF0121
:101E50008E919D018E3239F4CF010297DC018C9175
:101E60008083F90101C080833197EECFBFEF4B1A19
:101E70005B0A0BC00F5F1F4FF801AE16BF0628F4B8
:101E8000DF018E918083FD01F8CF81E3E1E0F0E096
:101E9000EC0FFD1FE20DF31D8083C156DF4FE8817B
:101EA000CF59D040EE2349F0F8018291803311F4EC
:101EB0008F01FACF8E3209F48F018820B1F1D80159
:101EC0008C92C801029657FE07C02DE211962C9302
:101ED00051944194510803C02BE2F80121838C01F5
:101EE000065F1F4F20E030E02F5F3F4FF801319633
:101EF000C2016AE070E00E945828805DD8018C938E
:101F00002B016115710511F08F01EECF22303105E3
:101F1000DCF3E21BF30B199781918E932150310969
:101F200012161306CCF309501109C256DF4FB881BF
:101F3000CE59D040BB2309F461C0E92DEC7F9E2E21
:101F4000CE56DF4FF881C259D0409F2ACD56DF4F81
:101F50002881C359D04020FB92F8CF56DF4F3881FB
:101F6000C159D04030FB93F8C057DF4F4881C0596A
:101F7000D04040FB94F8CC56DF4F5881C459D04034
:101F800050FB95F8C056DF4F8881C05AD04080FB87
:101F900096F8CB56DF4F9881C559D04090FB97F803
:101FA000292D237081E090E011F480E090E0910110
:101FB000281B390BF50140E35F01C8018E1B9F0B05
:101FC00082179307DCF44293F7CFC557DF4FB982EE
:101FD000A882CB58D040C456DF4FF983E883CC5950
:101FE000D040D12C0FE111E08CE1A82E81E0B82E79
:101FF00006C0D12C8E010A571F4F01C0D12C0A19DF
:102000001B09201631060CF440C0A92DAC7F9A2E76
:10201000CE56DF4FB881C259D0409B2ACD56DF4FF4
:10202000E881C359D040E0FB92F8CF56DF4FF881EA
:10203000C159D040F0FB93F8C057DF4F2881C059F9
:10204000D04020FB94F8CC56DF4F3881C459D040A3
:1020500030FB95F8C056DF4F4881C05AD04040FB56
:1020600096F8CB56DF4F5881C559D04050FB97F8B2
:102070007101E01AF10A292D237081E090E011F43A
:1020800080E090E0E81AF90A02C0E12CF12CCF566A
:10209000DF4F8881C159D040811122C031E0E31A5D
:1020A000F108F7FC1DC0C656DF4F68817981CA5917
:1020B000D04080E2C856DF4FE881F981C859D0404E
:1020C0000995C257DF4F28813981CE58D0402F5F04
:1020D0003F4FC257DF4F39832883CE58D040DECFE1
:1020E000492D4C7F942ECE56DF4F5881C259D04097
:1020F000952ACD56DF4F8881C359D04080FB92F896
:10210000CF56DF4F9881C159D04090FB93F8C0570C
:10211000DF4FA881C059D040A0FB94F8CC56DF4FC8
:10212000B881C459D040B0FB95F8C056DF4FE88164
:10213000C05AD040E0FB96F8CB56DF4FF881C55926
:10214000D040F0FB97F8892D837001F1813011F4B4
:102150008BE201C08DE2C656DF4F68817981CA5992
:10216000D040C856DF4FE881F981C859D040099561
:10217000C257DF4F28813981CE58D0402F5F3F4F63
:10218000C257DF4F39832883CE58D040D1100AC0C0
:102190003501C257DF4FA880B980CE58D040A6186D
:1021A000B70821C0C257DF4FC880D980CE58D04071
:1021B000AC18BD080150110917FD2DC0F501EC0D3B
:1021C000FD1D8491C656DF4F68817981CA59D04080
:1021D000C856DF4FE881F981C859D0400995FFEF13
:1021E000CF1ADF0AE7CF6501C60CD71C01501109D1
:1021F00017FD11C0C656DF4F68817981CA59D0409A
:10220000D3018D913D01C856DF4FE881F981C8594E
:10221000D0400995E8CFCF56DF4FF881C159D04063
:10222000FF2309F40CC921E0E21AF108F7FC07C901
:10223000C656DF4F68817981CA59D04080E2C856BE
:10224000DF4FE881F981C859D0400995FFEFCF1AD7
:10225000DF0AE9CFC257DF4F88819981CE58D0403D
:10226000CC55DF4F0FB6F894DEBF0FBECDBFDF9168
:10227000CF911F910F91FF90EF90DF90CF90BF9083
:10228000AF909F908F907F906F905F904F903F9016
:102290002F900895CF92DF92EF92FF920F931F93AA
:1022A000CF93DF931F92CDB7DEB77C01462F82E834
:1022B000860F9701265B3E4F6901823010F06B312B
:1022C00049F4F601608171818BE190E049830E94BD
:1022D00024094981D701A05BBE4F2C9111965C91D6
:1022E0001197842F90E0FC01E227EE0FFF1FEE52C2
:1022F000FC4F25913491052F10E0202731272D9395
:102300003C93F601608171810F90DF91CF911F9115
:102310000F91FF90EF90DF90CF900C9424092F92B3
:102320003F924F925F926F927F928F929F92AF9265
:10233000BF92CF92DF92EF92FF920F931F93CF93B2
:10234000DF93CDB7DEB7C455D1090FB6F894DEBF21
:102350000FBECDBF8C015C0126EBA21A2EEFB20A94
:102360004C014BEA841A4EEF940A7C0184EBE81A84
:102370008EEFF80AD5018D919C910E945A098F3FEA
:10238000BFEF9B0709F441C1F401208121110CC169
:102390008E37910509F0FAC0D7014D915C91F80193
:1023A000E25BFE4F1F014231510508F4E1C080811C
:1023B0009181883B904F09F0DBC0D801FE0138962F
:1023C000CE010E962D912695203209F420E021931E
:1023D000E817F907B9F7D80116968C9116978695E4
:1023E0008F708E871796FE013196CF0106962D913C
:1023F0002695203209F420E02193E817F907B9F770
:10240000F8013D96D8011D968C9186958F708F832B
:1024100029964FAC2997512C61E070E0808180FFB4
:1024200019C028965FAE289729964FAE299721812B
:10243000822F90E02B969FAF8EAF2B97039709F4D6
:1024400063C01F922F9384E991E09F938F938CE850
:1024500093E068C0B7E0B51520F366246394712C4F
:102460006C0E7D1E27E0529E600C711C1124CF0162
:10247000019663969FAF8EAF639780E090E0252D25
:1024800030E06396AEADBFAD6397DD906396BFAFAE
:10249000AEAF6397D694B0E2DB1202C0C12C01C08C
:1024A000CD2CD301A80FB91F1E96CC920196863071
:1024B000910539F737969081B7E0CB2EC29ED001B7
:1024C000C39EB00D1124CC24C394D12CCC0EDD1EA0
:1024D000AC0DBD1D892F86958F7054968C9397FFF8
:1024E00008C0CB0102C0880F991F2A95E2F7482A3D
:1024F00009C0DB0102C0AA0FBB1F2A95E2F79D01AC
:102500002095422253948ACF82812C968FAF2C97AC
:10251000803F99F01F928F9384E991E09F938F936E
:102520008BE493E09F938F930E945C250F900F9014
:102530000F900F900F900F901BC03396425051098F
:10254000C8018E1B9F0B480F591F60965FAF4EAF9F
:1025500060972E96FFAFEEAF2E97F801EE5AFE4F22
:102560000190F081E02D309719F0CE010196099588
:1025700081E0F801EC5AFE4F80838FEF9FEFD1018D
:102580008D939C93F70111821082F4CE8F379105C1
:1025900029F4F801EC5AFE4F1082ECCE8B319105F4
:1025A00019F481E08083E6CEF801EC5AFE4F2081D9
:1025B000222341F1D7012D913C912A34B1E03B0710
:1025C00000F5A9014F5F5F4FF70151834083F80188
:1025D000E20FF31F8083D801A25BBE4F2D913C9187
:1025E0001197F901E827FF27EE0FFF1FEE52FC4F6E
:1025F00085919491232F3327822793278D939C9342
:1026000001C01082D4011C92B5CEF5010081118168
:10261000D8011C968D919C911D97892B41F449E41A
:1026200051E069E373E08FE293E00E94DE25D80178
:102630001C96ED91FC911D97C8010995892B09F411
:1026400044C0F50100811181D8011C968D919C91A7
:102650001D97892B41F449E451E069E373E08FE26F
:1026600093E00E94DE25D8011C96ED91FC911D9708
:10267000C80109959F938F9389E991E09F938F9368
:1026800088EB93E09F938F930E945C25F501008176
:1026900011810F900F900F900F900F900F90D80115
:1026A0001E968D919C911F97892B41F442E551E034
:1026B0006DE173E080E193E00E94DE25D8011E9673
:1026C000ED91FC911F97C8010995CC5ADF4F0FB6C9
:1026D000F894DEBF0FBECDBFDF91CF911F910F9158
:1026E000FF90EF90DF90CF90BF90AF909F908F9032
:1026F0007F906F905F904F903F902F9008952F9212
:102700003F924F925F926F927F928F929F92AF9281
:10271000BF92CF92DF92EF92FF920F931F93CF93CE
:10272000DF93CDB7DEB72C970FB6F894DEBF0FBEA0
:10273000CDBF9C878B877B015A01288739871D83F2
:102740000C836115710541F448EF50E06EEF72E0C3
:1027500089EF92E00E94DE2522E0A216B10440F447
:1027600049EF50E067EE72E089ED92E00E94DE25CD
:102770004B845C8480EB481A8EEF580A8FEF9FEFF2
:10278000F201918380836B847C84F6EB6F1AFEEFF9
:102790007F0AF301608171818EE790E00E94240935
:1027A000C12CD12CC50101979F838E83CA14DB04F1
:1027B00009F468C021E029838E819F81C816D9065B
:1027C00009F01982F70101900020E9F78F0101500B
:1027D00011090E191F090730110510F006E010E06D
:1027E000C8018E0D9F1D9B838A8317018A819B815F
:1027F0002816390601F1F10121911F01822E912C39
:10280000C4012A870E94A8282A85892B51F42032E6
:1028100041F04BED50E064E972E08DE792E00E94F8
:10282000DE25C4010E94BC28682F660F8B859C851D
:102830000E944A11DBCF0630110599F0812C912CB2
:10284000E6E0F0E0E01BF10B8F018016910648F402
:1028500060E48B859C850E944A11FFEF8F1A9F0AC6
:10286000F4CF89818066F7016681660F682B8B85BE
:102870009C850E944A11FFEFCF1ADF0A27E0E20E83
:10288000F11C94CF63E08B859C850E944A1160EF18
:102890008B859C850E944A1108851985EC80FD80F6
:1028A000E00EF11E0E151F0541F0F80161918F0138
:1028B0008B859C850E944A11F5CFF20160811181C0
:1028C00060958B859C850E944A11612F60958B8550
:1028D0009C850E944A11F20180819181883B904F32
:1028E00041F042E151E067EC72E086EA92E00E943A
:1028F000DE25F301608171818EE790E02C960FB6A2
:10290000F894DEBF0FBECDBFDF91CF911F910F9125
:10291000FF90EF90DF90CF90BF90AF909F908F90FF
:102920007F906F905F904F903F902F900C94240970
:10293000EF92FF920F931F93CF93DF93EC018B01E4
:102940007A01009741F442E451E06BE672E087E6D9
:1029500092E00E94DE250115110541F443E451E0A7
:1029600065E572E08DE492E00E94DE2586E591E067
:10297000FE019C01119221503040E1F7FE01E65B1F
:10298000FE4F11830083FE01EE5AFE4FF182E0827A
:10299000FE01E05BFE4F8FEF9FEF91838083C25B70
:1029A000DE4F99838883DF91CF911F910F91FF9024
:1029B000EF90089566E773E00C94E41A78940E940F
:1029C000F60860E070E086E793E00E94460840E881
:1029D00055E260E070E086E793E00E94C80786E079
:1029E0008093C20060E070E08EEF94E00E945D1A78
:1029F0004AED54E16EEF74E088EA93E00E94981487
:102A00008FB7F894C090E305D090E405E090E50519
:102A1000F090E6058FBFC1E088EA93E00E948F1135
:102A20008091260281112EC086E793E00E94BA07AA
:102A3000882341F186E793E00E949607809329025C
:102A400090932A022091270230912802F901E55D36
:102A5000FD4FA9014F5F5F4F808350932802409341
:102A600027022934314010F0C09326028FB7F89422
:102A7000C090E305D090E405E090E505F090E60510
:102A80008FBF1BC08091270290912802892BA9F04B
:102A90002FB7F8948091E3059091E405A091E505A6
:102AA000B091E6052FBF8C199D09AE09BF090397A8
:102AB000A105B10514F0C093260280912602882357
:102AC00009F4AACF609127027091280228EA33E026
:102AD00046E753E08BE292E00E941B1C1092260214
:102AE000109228021092270297CFCF93DF93EC0128
:102AF0007093D9056093D8058630910544F041E282
:102B000050E06AED75E082ED95E00E94DE251092BE
:102B1000800089E18093810081E896E090938700AE
:102B2000809386008C2F806480937C0087B121E0A5
:102B300030E001C0220FCA95EAF7922F90958923C1
:102B400087B988B1892388B980917E00822B8093D0
:102B50007E0087E080937B008CEE80937A00DF918B
:102B6000CF9108951F920F920FB60F9211242F93B9
:102B70003F934F935F936F937F938F939F93AF9305
:102B8000BF93EF93FF9380E286BB609178007091D2
:102B90007900769567957695679560588091D80508
:102BA0009091D9050E9474178091E905882349F016
:102BB0008091D8059091D9050E944419807F886042
:102BC00007C08091E805882311F088E801C080E8FB
:102BD0008BB9FF91EF91BF91AF919F918F917F91B1
:102BE0006F915F914F913F912F910F900FBE0F907A
:102BF0001F901895AF92BF92CF92DF92EF92FF9203
:102C00000F931F93CF93DF936C01EB017A01DC01EB
:102C100050960D911D912D913C9153970D341B446D
:102C20002345364441F04EE650E061E076E08BEE1D
:102C300095E00E94DE255E01CE018E0D9F1DF601FE
:102C4000EB57FF4FA816B90671F4C5018C1B9D0BFD
:102C5000DF91CF911F910F91FF90EF90DF90CF9078
:102C6000BF90AF9008956FB7F89440815181228151
:102C700033816FBF4217530741F32FB7F894C090C9
:102C8000E305D090E405E090E505F090E6052FBF60
:102C90006FB7F89440815181228133816FBF421711
:102CA0005307A9F44FB7F8940091E3051091E40598
:102CB0002091E5053091E6054FBF0C191D092E093D
:102CC0003F09101611061206130614F7BECF6FB790
:102CD000F89420813181468157812417350719F4F2
:102CE0004481558105C020813181A9014F5F5F4F2B
:102CF00051834083D9012C916FBFD5012D935D0184
:102D0000A1CF6F927F928F929F92AF92BF92CF92FC
:102D1000DF92EF92FF920F931F93CF93DF93EC011B
:102D20008B017A0188899989AA89BB898D349B4452
:102D3000A345B64441F04EE650E061E076E08BEE0C
:102D400095E00E94DE25F801A8014E0D5F1D992433
:102D50009394BB24B3943E0187E7680E711C20E472
:102D600030E065E370E088E0E82EF12CE417F50729
:102D700009F44EC0AFB6F894CFA4D8A88BA99CA9EB
:102D8000C816D90639F4C9A8DAA88DA99EA9C8160B
:102D9000D90669F0C9A8DAA88FA598A9019788244F
:102DA0008394C816D90609F0812C882D01C081E0D2
:102DB000AFBE80FDDFCFD190AFB6F89489A99AA9B4
:102DC000DC01DC92C9A8DAA88DA99EA9C816D9068B
:102DD00019F48BA99CA903C089A99AA901969AAB59
:102DE00089ABAFBED3018C9181110CC03EA72DA73A
:102DF0001CA61BA61AA69C92299A7BA36AA35B9A7F
:102E0000B092E9058FB7F894FDA2ECA28FBFAECFC8
:102E1000CF01801B910BDF91CF911F910F91FF90FC
:102E2000EF90DF90CF90BF90AF909F908F907F906A
:102E30006F900895CF93DF93EC01488959896A898F
:102E40007B894D345B446345764441F04EE650E067
:102E500061E076E08BEE95E00E94DE25C958DF4FF9
:102E600088818111FDCF80E090E0DF91CF910895BE
:102E7000CF93DF93EC01488959896A897B894D3466
:102E80005B446345764441F04EE650E061E076E015
:102E90008BEE95E00E94DE252FB7F894C852DF4FE5
:102EA000888199812FBFDF91CF910895CF93DF93D0
:102EB000EC01488959896A897B894D345B446345B3
:102EC000764441F04EE650E061E076E08BEE95E02E
:102ED0000E94DE258FB7F894C852DF4F19821882FE
:102EE0008FBFDF91CF910895EF92FF920F931F93C1
:102EF000CF93DF93FC018C0101531F4FD8014D91FB
:102F00005C91DC01A353BF4F4D935C93DC01A85847
:102F1000BF4F8D919C91119716962D913C911797CB
:102F20008217930729F414962D913C91159706C0AA
:102F30008D919C9111979C012F5F3F4F11963C936F
:102F40002E93EC01288126029001112435952795B6
:102F500035952795E801398328837F01D3EDED0E60
:102F6000F11CE701888199818F010F521F4FE80101
:102F70009983888395958795840F951F820F931F5A
:102F8000E70199838883AF014B525F4F21E0181608
:102F900019060CF020E0EA018881880F822B8883D3
:102FA00012968D919C911397EC01688312962D9146
:102FB0003C91139716968D919C9117972817390776
:102FC00029F414968D919C91159705C012968D91B8
:102FD0009C911397019613969C938E931297DA0106
:102FE0009C91892F8695869589278370DF01AA5247
:102FF000BF4F833039F48C91803214F48F5F01C05D
:1030000081508C938C91885F8C9380340CF435C103
:103010008F738C93DF01A952BF4F8C91880F9770EB
:103020002BEF290F233010F0933009F481608C933B
:103030009C91892F8695892780958170968D990F0F
:10304000892B868F8E3709F04EC0DF01AB57BF4FFB
:103050002D913C91119714968D919C91159728175D
:10306000390759F412962D913C91139716968D912C
:103070009C9117972817390779F012962D913C915A
:1030800013978D919C911197019741E0281739076B
:1030900009F040E0842F01C081E080FDDDC0129680
:1030A000CD91DC9113978EE7888312962D913C91F8
:1030B000139716968D919C9117972817390729F425
:1030C00014968D919C91159705C012968D919C91A7
:1030D0001397019613969C938E93129781E081A388
:1030E0002A9A41E0BCC0982F9F779F3719F411A20C
:1030F0002A98C3C091A1992309F4BFC0982F9F7348
:103100009E3309F4BAC080FF03C080A1806880A309
:10311000878D8F5F878F90A1883008F4ACC0DF0166
:10312000AB57BF4F82E8890F823018F09B3109F00E
:103130004BC02D913C91119714968D919C911597B0
:103140002817390759F412962D913C91139716962A
:103150008D919C9117972817390779F012962D9128
:103160003C9113978D919C911197019741E02817FD
:10317000390709F040E0842F01C081E080FD20C0C4
:103180001296CD91DC9113978BE1888312962D9145
:103190003C91139716968D919C9117972817390794
:1031A00029F414968D919C91159705C012968D91D6
:1031B0009C911397019613969C938E93129704C03B
:1031C00011A22A9840E001C041E02D913C91119755
:1031D00014968D919C9115972817390759F41296DA
:1031E0002D913C91139716968D919C9117972817C6
:1031F000390779F012962D913C9113978D919C91FE
:103200001197019751E02817390709F050E0852FF1
:1032100001C081E080FD20C080A11296CD91DC919B
:103220001397888312962D913C91139716968D9142
:103230009C9117972817390729F414968D919C9122
:10324000159705C012968D919C9113970196139630
:103250009C938E93129703C011A22A9840E010A26B
:10326000178E41110AC0E852FF4F80819181816021
:103270009183808302C0969590A3DF91CF911F9197
:103280000F91FF90EF900895DC0196968C919697A0
:103290008111EAC098968C9198978111A0C09F9651
:1032A0002D913C91D097D1968D919C91D2972817D2
:1032B000390739F494968D919C919597892B09F44F
:1032C0005CC099968C919997811103C09A961C9233
:1032D0009A9781E099968C93999792968D919C916B
:1032E0009397009789F59F962D913C91D097D19611
:1032F0008D919C91D2972817390751F494968D910E
:103300009C919597019795969C938E93949721C045
:103310009F96ED91FC91D097D5968D919C91D697E3
:10332000E817F90729F4D3968D919C91D49706C09C
:103330009F96ED91FC91D097CF010196D0969C93EA
:103340008E939F97808106C0019793969C938E934E
:1033500092978EE797968C93979797968C919797DD
:103360008B3199F59F962D913C91D097D1968D9167
:103370009C91D2972817390749F45B981092E90578
:10338000A958BF4F1C92299880E008959F96ED910F
:10339000FC91D097D5968D919C91D697E817F90717
:1033A00029F4D3968D919C91D49706C09F96ED9168
:1033B000FC91D097CF010196D0969C938E939F97C6
:1033C000808197968C93979706C08E57823018F419
:1033D00099961C92999781E098968C9398979996D4
:1033E0002C9199979D968D919C919E972223A9F05F
:1033F0009A962C919A97253080F09A961C929A97DB
:103400008034910519F485E790E002C080E490E0F3
:103410009E969C938E939D9723C098963C919897E7
:1034200097962C919797232341F09A968C919A978F
:103430008F5F9A968C939A970FC09A961C929A9740
:103440008034910519F485E790E002C080E490E0B3
:103450009E969C938E939D97330F98963C93989746
:1034600088E096968C9396979D96ED91FC919E9709
:103470009B968D919C919C97E80FF91F9F0131704D
:103480009C963C932E939B9796968C919697815001
:1034900096968C93FF27E038F10530F08FEF90E09F
:1034A000AC014E1B5F0BFA01E25FF94F84912F3F95
:1034B000310511F008F080950895CF93DF93EC016A
:1034C000CB012AEDFE0111922A95E9F77D8F6C8FD1
:1034D00020E430E03EA72DA79E0120583F4FFE017B
:1034E000E858FF4F3583248333832283318320833D
:1034F0009E012C573F4F378326839E0123573F4F12
:10350000DE01AB57BF4F15963C932E93149713963D
:103510003C932E93129711963C932E939E01245325
:103520003F4F17963C932E9316979E01295C3F4F71
:103530003CAB2BAB3AAB29AB38AB2FA79E012A583B
:103540003F4F3EAB2DAB24E030E0A281B3811C9213
:1035500062817381468157816417750719F444812C
:10356000558104C0428153814F5F5F4F5383428333
:10357000215031092115310541F7BE010E94751511
:103580008AB1886F8AB9219A229A4DE45BE463E597
:1035900076E4488B598B6A8B7B8B81E896E19B8321
:1035A0008A838AEF95E1998388838AE197E19B87F3
:1035B0008A8788E397E19D878C8786E597E19F87D7
:1035C0008E87DF91CF9108958F929F92AF92BF9295
:1035D000CF92DF92EF92FF920F931F93CF93DF93DF
:1035E000EC014B01809147018823F1F08091430168
:1035F000882329F064EA71E0C4010E9498098E8151
:103600001F928F93DF93CF938AEA91E09F938F93DA
:103610009F928F920E948609EDB7FEB738960FB63B
:10362000F894FEBF0FBEEDBF80914601882339F1AB
:1036300080914301882361F085EB91E09F938F9304
:103640009F928F920E9486090F900F900F900F907B
:103650008D851F928F93CE0107969F938F938AEA51
:1036600091E09F938F939F928F920E9486098DB7CE
:103670009EB708960FB6F8949EBF0FBE8DBF80917F
:103680004501811105C080914401811137C05CC0A2
:1036900080914301882329F06BEB71E0C4010E9403
:1036A00098098E01025F1F4FE12CF12C5E0196E418
:1036B000A90EB11C8AEAC82E81E0D82EF5018081BE
:1036C00090E0E816F906FCF6F80186811F928F93C8
:1036D0001F930F93DF92CF929F928F920E94860941
:1036E000FFEFEF1AFF0A095F1F4F8DB79EB70896CD
:1036F0000FB6F8949EBF0FBE8DBFE0CF80914301FF
:10370000882329F062EC71E0C4010E949809FE014F
:10371000E55BFF4F81818F9380818F93C35BDF4F88
:1037200089818F9388818F9329EC31E03F932F9388
:103730009F928F920E9486098DB79EB708960FB60A
:10374000F8949EBF0FBE8DBF6EEC71E0C401DF9197
:10375000CF911F910F91FF90EF90DF90CF90BF908E
:10376000AF909F908F900C9498090F931F939C019A
:10377000CA0146E0E7E3F1E0A6E0B6E001900D9271
:103780004A95E1F74091DA0540930C0646E0EDE3F7
:10379000F1E0A4E1B6E001900D924A95E1F7409185
:1037A000DC0540931A0646E0E1E3F1E0ADE0B6E067
:1037B00001900D924A95E1F740912F014093130635
:1037C00046E0E9E2F1E0ABE1B6E001900D924A9506
:1037D000E1F7409127014093210647E0E6E0F6E05B
:1037E000AAEEB5E001900D924A95E1F747E0E4E1D9
:1037F000F6E0A1EFB5E001900D924A95E1F747E0C0
:10380000EDE0F6E0A8EFB5E001900D924A95E1F702
:1038100047E0EBE1F6E0AFEFB5E001900D924A959D
:10382000E1F78B0144E050E06AEE75E00E947F13FF
:103830001F910F910895EF92FF920F931F93CF93D3
:10384000DF93EC018B0179018091DE05882361F023
:1038500081ED91E09F938F935F934F930E94860930
:103860000F900F900F900F900115110509F40BC1E7
:103870008881813291F40230110508F404C1B80145
:1038800061507109A701CE010196DF91CF911F917F
:103890000F91FF90EF900C94B51B8336F9F4043030
:1038A000110508F4F0C0EDE3F1E081E090E0DE0105
:1038B000A80FB91F2C91222331F02A3021F02D308E
:1038C00011F0208301C01082019631968017910774
:1038D00009F4D9C08730910551F7D5C08436F9F481
:1038E0000430110508F4CFC0E7E3F1E081E090E097
:1038F000DE01A80FB91F2C91222331F02A3021F0CC
:103900002D3011F0208301C010820196319680176E
:10391000910709F4B8C08730910551F7B4C08133DD
:10392000F9F40230110508F4AEC0E1E3F1E081E002
:1039300090E0DE01A80FB91F2C91222331F02A302C
:1039400021F02D3011F0208301C0108201963196B4
:103950008017910709F497C08730910551F793C0FC
:103960008233F9F40230110508F48DC0E9E2F1E088
:1039700081E090E0DE01A80FB91F2C91222331F0E5
:103980002A3021F02D3011F0208301C010820196E1
:1039900031968017910709F476C08730910551F769
:1039A00072C0833771F50330110508F46CC089814A
:1039B000833639F48A8190E0C0979093DD05809337
:1039C000DC058981843639F48A8190E0C097909330
:1039D000DB058093DA058981813339F48A8190E0AF
:1039E000C0979093300180932F018981823309F031
:1039F0004AC08A8190E0C097909328018093270164
:103A000042C0803709F03FC003301105E0F18981E1
:103A1000833751F48A81813321F481E08093470117
:103A200032C0109247012FC0843651F48A8181330D
:103A300021F481E08093460126C01092460123C004
:103A4000803751F48A81813321F481E080934501EC
:103A50001AC01092450117C08D3651F48A81813306
:103A600021F481E0809344010EC0109244010BC008
:103A7000893649F48A81813321F481E080934301BE
:103A800002C010924301DF91CF911F910F91FF90DF
:103A9000EF9008952F923F924F925F926F927F9294
:103AA0008F929F92AF92BF92CF92DF92EF92FF924E
:103AB0000F931F93CF93DF93CDB7DEB7C45AD109CD
:103AC0000FB6F894DEBF0FBECDBFC856DF4F998347
:103AD0008883C859D040C656DF4F79836883CA5956
:103AE000D040C456DF4F59834883CC59D040590148
:103AF000C257DF4F19821882CE58D0409E012F5FE7
:103B00003F4FC957DF4F39832883C758D040AE0194
:103B10004A575F4FC757DF4F59834883C958D04032
:103B2000C856DF4F08811981C859D0400F5F1F4F19
:103B3000C856DF4FE881F981C859D0408491853259
:103B400091F1882309F448C7C456DF4F6881798111
:103B5000CC59D040C656DF4FE881F981CA59D040D0
:103B60000995C257DF4FE880F980CE58D040FFEF6B
:103B7000EF1AFF0AC557DF4FB982A882CB58D04051
:103B8000C856DF4F19830883C859D040C257DF4F4A
:103B9000F982E882CE58D040C557DF4FA880B9805F
:103BA000CB58D040BDCFF8018491853259F5C85625
:103BB000DF4F28813981C859D0402E5F3F4FC8560A
:103BC000DF4F39832883C859D040C456DF4F6881FE
:103BD0007981CC59D040C656DF4FE881F981CA5966
:103BE000D0400995C257DF4FE880F980CE58D040C9
:103BF000FFEFEF1AFF0AC557DF4FB982A882CB58F3
:103C0000D040C4CFC256DF4F1882CE59D040C357E0
:103C1000DF4F1882CD58D040C057DF4F1882C059AF
:103C2000D040CF56DF4F1882C159D040F8012491BF
:103C3000C80101962B3209F458C060F42032E9F033
:103C4000233209F05AC0F1E0C357DF4FF883CD5853
:103C5000D04051C02D3251F0203309F04EC021E048
:103C6000C256DF4F2883CE59D04045C0F1E0C0573F
:103C7000DF4FF883C059D0403EC0232D2C7F322E19
:103C8000CF56DF4F3881C159D040332ACE56DF4F4F
:103C90004881C259D04040FB32F8C057DF4F5881AD
:103CA000C059D04050FB33F820FA34F8CD56DF4FDE
:103CB000A881C359D040A0FB35F8C357DF4FB88166
:103CC000CD58D040B0FB36F8CC56DF4FE881C45910
:103CD000D040E0FB37F8232D237069F441E0CF5644
:103CE000DF4F4883C159D04006C031E0CF56DF4F87
:103CF0003883C159D0408C0199CFC357DF4F5881C9
:103D0000CD58D040C056DF4F5883C05AD040F8013C
:103D100024912A3221F0612C712C3AE025C09501C2
:103D20002E5F3F4FD5016D907C9077FE09C0719456
:103D300061947108B1E0C057DF4FB883C059D040DB
:103D40008C01590116C02A33A0F40F5F1F4FFC01EC
:103D50008491A301349F3001359F700C112450E3EE
:103D6000651A7108680E711CC801F801249120338E
:103D700050F7C057DF4FF881C059D040FF2329F0DA
:103D8000C256DF4F1882CE59D040F80184918E324E
:103D900049F5319684918A3229F08F01412C512CBA
:103DA0003AE01AC0D5014D905C900E5F1F4FF501AF
:103DB00032965F011AC02A33C0F40F5F1F4FFC0117
:103DC0008491A201349F2001359F500C112450E3AF
:103DD000451A5108480E511CC801F801249120339E
:103DE00050F703C044244A94542CF8012491C8018C
:103DF0000196283699F018F42C3439F017C02C3677
:103E000021F02A3799F4212C02C0222423948C011A
:103E1000CD56DF4F1882C359D0400EC08C01F1E05F
:103E2000CD56DF4FF883C359D04005C0CD56DF4F84
:103E30001882C359D040212C98012F5F3F4FC8569C
:103E4000DF4F39832883C859D040F801D490C95630
:103E5000DF4FD882C759D040F5E6DF1609F402C219
:103E6000FD15ECF023E5D21609F453C02D1564F0CE
:103E700035E4D31609F4F6C147E4D41609F4E1C1D8
:103E8000DD2009F46FC42AC053E6D51671F15D1523
:103E90000CF4C6C088E5D81609F48DC01FC090E7A1
:103EA000D91609F471C09D1564F0A7E6DA1609F475
:103EB000C8C1DA160CF4D1C1B9E6DB1609F4B0C0FA
:103EC0000DC0E5E7DE1609F476C0F8E7DF1609F461
:103ED0006DC023E7D21202C0F12C1DC0C557DF4FC1
:103EE000B982A882CB58D04049C4A5014E5F5F4F2C
:103EF000C557DF4F59834883CB58D040D5018C91AB
:103F00008983F12C8E010E5F1F4FFE0131964F0108
:103F100043C4FF24F39495012E5F3F4FC557DF4FF5
:103F200039832883CB58D040D5018D909C90811443
:103F3000910421F4ACE48A2EA1E09A2E57FE04C02D
:103F4000F0E14F2EF7E25F2E8401FF20C1F0F8016F
:103F50008491882309F420C4C8018819990984151B
:103F600095050CF019C40F5F1F4FF1CFC8018819D8
:103F70009909841595050CF00FC40F5F1F4FD801E8
:103F80008C918111F3CF08C4F5013296C557DF4FEC
:103F9000F983E883CB58D040D5016D917C9180E0C6
:103FA00090E0EBE6EE2EE1E0FE2E26C07BE7E72E6A
:103FB00071E0F72E04C06BE6E62E61E0F62E2220BB
:103FC00071F0F5013496C557DF4FF983E883CB587C
:103FD000D040D5016D917D918D919C910DC0C50111
:103FE0000296F50160817181C557DF4F99838883FF
:103FF000CB58D04080E090E021E0CE56DF4F2883C0
:10400000C259D04035E7D31205C0CE56DF4F1882D3
:10401000C259D040CF56DF4F1882C159D0403EC060
:10402000222079F0A5014C5F5F4FC557DF4F5983C0
:104030004883CB58D040D5016D917D918D919C9155
:104040000FC0F5013296C557DF4FF983E883CB588F
:10405000D040D5016D917C91882777FD8095982F70
:1040600097FF13C090958095709561957F4F8F4F06
:104070009F4FCE56DF4F1882C259D040B2E0CF5684
:10408000DF4FB883C159D04005C0CE56DF4F1882EC
:10409000C259D0405BE6E52E51E0F52EE1E0CC566A
:1040A000DF4FE883C459D040611571058105910542
:1040B00029F4CC56DF4F1882C459D0404114510422
:1040C00041F4CC56DF4FF881C459D040FF2309F4A6
:1040D00076C0CE56DF4F2881C259D0408E010A5794
:1040E0001F4F2130A9F02AE030E040E050E00E946C
:1040F0006C28F701E60FF71F8081D8018E938D01A0
:10410000B901CA01611571058105910561F715C0F5
:10411000FB01EF70FF27EE0DFF1D2081F8012293B8
:104120008F0144E096958795779567954A95D1F7E5
:10413000611571058105910559F757FE43C0C256B7
:10414000DF4FF881CE59D040FF23E1F1232D2C7FA2
:10415000322ECF56DF4F3881C159D040332ACE5648
:10416000DF4F4881C259D04040FB32F8C057DF4F83
:104170005881C059D04050FB33F820FA34F8CD565E
:10418000DF4F8881C359D04080FB35F8C357DF4FDC
:104190009881CD58D04090FB36F8CC56DF4FA8819F
:1041A000C459D040A0FB37F8232D237081E090E064
:1041B00011F480E090E02301481A590A03C08E01EF
:1041C0000A571F4FC757DF4F88819981C958D04080
:1041D000801B910BF80120E34F01841595051CF419
:1041E00022930196F9CFC357DF4FB881CD58D04005
:1041F000BB23A1F0CC56DF4FE881C459D040EE2359
:1042000069F08D2D8F7D883549F4F4013197D08286
:10421000F2E08F1A910880E3D4018C93C957DF4FE5
:10422000E881F981C758D0408E169F0608F0AEC2CB
:1042300047EB52E061EA76E08EE896E00E94DE25E8
:10424000A5C2DA94DA94C956DF4FD882C759D04054
:1042500011E04114510469F006C0C956DF4F1882BD
:10426000C759D04010E057FE07C026E0422E512C1F
:1042700003C044244394512C95012C5F3F4FC557F4
:10428000DF4F39832883CB58D040D501CD90DD90C6
:10429000ED90FC9020E030E0A901C701B6010E943A
:1042A0007E2687FF0AC0F7FAF094F7F8F094B2E0A0
:1042B000CF56DF4FB883C159D040C156DF4F188366
:1042C000CF59D04088248394912C8C0E9D1E860C4F
:1042D000971C20E030E040E85FE3C701B6010E9490
:1042E000CD2787FD32C0A12CB12C27EB33E44AEB5C
:1042F00051E5C701B6010E94CD2787FD0EC029EF09
:1043000032E045E150E5C701B6010E9482266B010B
:104310007C01EAE0AE0EB11CE8CF20E030E040E2E4
:1043200051E4C701B6010E94CD2787FD49C020E0B6
:1043300030E040E251E4C701B6010E9482266B01E1
:104340007C01FFEFAF1ABF0AE8CF20E030E0A901FF
:10435000C701B6010E947E26A12CB12C882381F1D1
:104360002FEF36EE4BED5EE2C701B6010E947E26CE
:10437000181674F029EF32E045E150E5C701B601A7
:104380000E94D1276B017C012AE0A21AB108E8CF74
:1043900020E030E040E85FE3C701B6010E947E26DE
:1043A00087FF0EC020E030E040E251E4C701B601D3
:1043B0000E94D1276B017C0131E0A31AB108E8CF3C
:1043C000112321F1A414B50464F44CEFA4164FEFAB
:1043D000B4063CF04A185B08C956DF4F1882C7592B
:1043E000D04051E0451A510881E0C357DF4F988112
:1043F000CD58D0409827C156DF4F9883CF59D04031
:10440000A1E0C357DF4FA883CD58D040C956DF4F36
:10441000B881C759D040B1114CC0B7FE3EC080E34F
:10442000E1E0F0E0EC0FFD1FE60DF71D8083411485
:10443000510461F4C357DF4FE881CD58D040E111FA
:1044400005C0F401319680E090E007C0F401329697
:104450008EE2D40111968C93C20195012F5F3F4FDC
:10446000280F391F40E38F018217930729F0009727
:1044700019F041930197F7CF920120953095A2163C
:10448000B3060CF4D6C02C01E1E0F0E0CB56DF4FD0
:10449000F983E883C559D0405CC0222733272A1905
:1044A0003B09CB56DF4F39832883C559D04084015F
:1044B00050C08401CB56DF4F19821882C559D040B5
:1044C00048C0C701B6010E94EA26CF55DF4F688376
:1044D00079838A839B83C15AD040CF55DF4F48816F
:1044E0005981C15AD040BA01882777FD8095982F0D
:1044F0000E941D279B01AC01C701B6010E9419262D
:1045000020E030E040E251E40E94D1276B017C01C1
:1045100098012F5F3F4FCF55DF4F8881C15AD04060
:10452000805DD8018C93CB56DF4F88819981C55926
:10453000D0400196CB56DF4FE881F981C559D04074
:10454000EF2B91F0CB56DF4F99838883C559D0402C
:104550008901CB56DF4F28813981C559D040421699
:1045600053060CF0AECF14C04114510439F4C357B4
:10457000DF4FF881CD58D040FF2339F098012E5FEE
:104580003F4FEEE2D8011196EC9381E090E0DACF54
:1045900020E030E040EA50E4C701B6010E94CD2798
:1045A00087FD47C0F80181E090E030E322912E3290
:1045B00051F0820F8A3321F0808380E090E003C0C5
:1045C000308381E090E08E169F0680F3892B89F17D
:1045D000C956DF4F3881C759D0403323B9F0F801AD
:1045E0008E169F0678F4DF018E919D018E3239F48C
:1045F000CF010297DC018C918083F90101C0808397
:104600003197EECFBFEFAB1ABB0A0BC00F5F1F4F46
:10461000F8018E169F0628F4DF018E918083FD013C
:10462000F8CF81E3E1E0F0E0EC0FFD1FE60DF71DB0
:104630008083C156DF4FE881CF59D040EE2349F047
:10464000F8018291803311F48F01FACF8E3209F490
:104650008F01C956DF4FF881C759D040FF23B9F108
:10466000D801FC93C8010296B7FE07C02DE211964F
:104670002C93B194A194B10804C02BE2D8011196F7
:104680002C938C01065F1F4F20E030E02F5F3F4FDF
:10469000F8013196C5016AE070E00E945828805DFB
:1046A000D8018C935B016115710511F08F01EECF7C
:1046B00022303105DCF3E21BF30B199781918E93C5
:1046C0002150310912161306CCF309501109C256B4
:1046D000DF4FB881CE59D040BB2309F45CC0E32D35
:1046E000EC7F3E2ECF56DF4FF881C159D0403F2A94
:1046F000CE56DF4F2881C259D04020FB32F8C05738
:10470000DF4F3881C059D04030FB33F820FA34F8FD
:10471000CD56DF4F4881C359D04040FB35F8C056D5
:10472000DF4F5881C05AD04050FB36F8CC56DF4F8F
:104730008881C459D04080FB37F8232D237081E055
:1047400090E011F480E090E09301281B390BF40114
:1047500040E34F01C8018E1B9F0B82179307DCF4C7
:104760004293F7CFC557DF4FB982A882CB58D040CC
:10477000C856DF4F19830883C859D040F12C0BE489
:1047800011E088E4882E81E0982E06C0F12C8E017D
:104790000A571F4F01C0F12C08191909601671063C
:1047A000DCF1932D9C7F392ECF56DF4FA881C15964
:1047B000D0403A2ACE56DF4FB881C259D040B0FB24
:1047C00032F8C057DF4FE881C059D040E0FB33F8E2
:1047D00020FA34F8CD56DF4FF881C359D040F0FBB2
:1047E00035F8C056DF4F2881C05AD04020FB36F83C
:1047F000CC56DF4F3881C459D04030FB37F86301C5
:10480000C01AD10A232D237081E090E011F480E0DA
:1048100090E0C81AD90A02C0C12CD12CC057DF4F72
:104820004881C059D040411122C031E0C31AD1089B
:10483000D7FC1DC0C456DF4F68817981CC59D04068
:1048400080E2C656DF4FE881F981CA59D040099508
:10485000C257DF4F28813981CE58D0402F5F3F4F5C
:10486000C257DF4F39832883CE58D040DECF432D47
:104870004C7F342ECF56DF4F5881C159D040352A56
:10488000CE56DF4F8881C259D04080FB32F8C057E6
:10489000DF4F9881C059D04090FB33F820FA34F8AC
:1048A000CD56DF4FA881C359D040A0FB35F8C05684
:1048B000DF4FB881C05AD040B0FB36F8CC56DF4F3E
:1048C000E881C459D040E0FB37F8832D837001F1B3
:1048D000813011F48BE201C08DE2C456DF4F688154
:1048E0007981CC59D040C656DF4FE881F981CA5949
:1048F000D0400995C257DF4F28813981CE58D0402A
:104900002F5F3F4FC257DF4F39832883CE58D040A7
:10491000F11009C0C257DF4FA880B980CE58D040EF
:10492000A818B90822C0C257DF4FE880F980CE58D6
:10493000D0405401AE18BF080150110917FD2DC019
:10494000F501EE0DFF1D8491C456DF4F688179811A
:10495000CC59D040C656DF4FE881F981CA59D040C2
:104960000995FFEFEF1AFF0AE7CF7501E80CF91C74
:104970000150110917FD11C0C456DF4F68817981BC
:10498000CC59D040D4018D914D01C656DF4FE881FE
:10499000F981CA59D0400995E8CFC057DF4FF88157
:1049A000C059D040FF2309F4F1C821E0C21AD10850
:1049B000D7FCECC8C456DF4F68817981CC59D04010
:1049C00080E2C656DF4FE881F981CA59D040099587
:1049D000FFEFEF1AFF0AE9CFC257DF4F88819981B5
:1049E000CE58D040CC55DF4F0FB6F894DEBF0FBE87
:1049F000CDBFDF91CF911F910F91FF90EF90DF908E
:104A0000CF90BF90AF909F908F907F906F905F906E
:104A10004F903F902F9008959091C00095FFFCCF4C
:104A20008A3041F09091C00090649093C0008093D0
:104A3000C60008959091C00090649093C0009DE0DE
:104A40009093C6009091C00095FFFCCFEBCFCF9321
:104A50009B01C091C1004091C10048604093C100DA
:104A60004091C1004F794093C10040E050E06CE0BC
:104A700075E20E944A1D8091C00086FFFCCFC09362
:104A8000C100CF910895CF93C091C1009091C10012
:104A900098609093C1009091C1009F799093C1005C
:104AA00060E070E00E940C258091C00086FFFCCF82
:104AB000C093C100CF910895CF93DF93CDB7DEB7F8
:104AC000FE01359681919191BF010E942725DF91CA
:104AD000CF9108951F93CF93DF931091C100209140
:104AE000C10028602093C1002091C1002F7920933C
:104AF000C100FC018491EF012196882331F060E030
:104B000070E00E940C25FE01F5CF8091C00086FF69
:104B1000FCCF1093C100DF91CF911F910895AF9208
:104B2000BF92CF92DF92EF92FF920F931F93CF939A
:104B3000DF936C0185E0E82EF12C00E117E2C0E084
:104B4000D0E09AE0A92EB12CC601B8010E945828E5
:104B50006C016115710529F4209719F401301105D4
:104B600029F480E3860F0E9443252196C801B501F0
:104B70000E9458288B0181E0E81AF108E114F10441
:104B800019F7CE01DF91CF911F910F91FF90EF9018
:104B9000DF90CF90BF90AF900895CF93DF93EB015C
:104BA0000E946A258AE30E944325CE010E948F2538
:104BB00080ED96E0DF91CF910C946A25CF93DF933F
:104BC000EC01CB01BA010E94CD2583ED96E00E9455
:104BD0006A25CE010E946A258AE00E94432581E071
:104BE00090E0DF91CF9108950F931F93CF93DF93C0
:104BF000182F092FEB01B901CA010E94CD2582ECC3
:104C000096E00E946A25CE010E946A250F931F93A9
:104C100089EB96E09F938F930E945C250F900F90F5
:104C20000F900F9081E090E0DF91CF911F910F9155
:104C300008955058BB27AA270ED075C166D130F011
:104C40006BD120F031F49F3F11F41EF45BC10EF4E0
:104C5000E095E7FB51C1E92F77D180F3BA176207DE
:104C600073078407950718F071F49EF58FC10EF451
:104C7000E0950B2EBA2FA02D0B01B90190010C016C
:104C8000CA01A0011124FF27591B99F0593F50F484
:104C9000503E68F11A16F040A22F232F342F4427DC
:104CA000585FF3CF469537952795A795F0405395D4
:104CB000C9F77EF41F16BA0B620B730B840BBAF0A4
:104CC0009150A1F0FF0FBB1F661F771F881FC2F70F
:104CD0000EC0BA0F621F731F841F48F48795779523
:104CE0006795B795F7959E3F08F0B3CF9395880FDA
:104CF00008F09927EE0F979587950895D9D008F475
:104D000081E008950CD00FC107D140F0FED030F003
:104D100021F45F3F19F0F0C0511139C1F3C014D133
:104D200098F39923C9F35523B1F3951B550BBB2772
:104D3000AA2762177307840738F09F5F5F4F220F1F
:104D4000331F441FAA1FA9F333D00E2E3AF0E0E818
:104D500030D091505040E695001CCAF729D0FE2F64
:104D600027D0660F771F881FBB1F261737074807F6
:104D7000AB07B0E809F0BB0B802DBF01FF279358AC
:104D80005F4F2AF09E3F510568F0B6C000C15F3FFB
:104D9000ECF3983EDCF3869577956795B795F79594
:104DA0009F5FC9F7880F911D9695879597F908958C
:104DB000E1E0660F771F881FBB1F62177307840728
:104DC000BA0720F0621B730B840BBA0BEE1F88F737
:104DD000E095089504D06894B111D9C00895BCD06D
:104DE00088F09F5790F0B92F9927B751A0F0D1F0D4
:104DF000660F771F881F991F1AF0BA95C9F712C05E
:104E0000B13081F0C3D0B1E00895C0C0672F782FD2
:104E10008827B85F39F0B93FCCF3869577956795C9
:104E2000B395D9F73EF490958095709561957F4F35
:104E30008F4F9F4F0895E89409C097FB3EF49095DB
:104E40008095709561957F4F8F4F9F4F9923A9F063
:104E5000F92F96E9BB279395F695879577956795F2
:104E6000B795F111F8CFFAF4BB0F11F460FF1BC036
:104E70006F5F7F4F8F4F9F4F16C0882311F096E9C9
:104E800011C0772321F09EE8872F762F05C0662377
:104E900071F096E8862F70E060E02AF09A95660F30
:104EA000771F881FDAF7880F9695879597F90895E9
:104EB000990F0008550FAA0BE0E8FEEF161617062B
:104EC000E807F907C0F012161306E407F50798F093
:104ED000621B730B840B950B39F40A2661F0232BAC
:104EE000242B252B21F408950A2609F4A140A69528
:104EF0008FEF811D811D089597F99F6780E870E00D
:104F000060E008959FEF80EC089500240A9416163F
:104F1000170618060906089500240A9412161306A7
:104F2000140605060895092E0394000C11F4882335
:104F300052F0BB0F40F4BF2B11F460FF04C06F5F51
:104F40007F4F8F4F9F4F089557FD9058440F551F27
:104F500059F05F3F71F04795880F97FB991F61F0FB
:104F60009F3F79F087950895121613061406551F72
:104F7000F2CF4695F1DF08C0161617061806991FDE
:104F8000F1CF86957105610508940895E894BB27D3
:104F900066277727CB0197F908958ADF08F48FEF0A
:104FA00008950BD0C0CFB1DF28F0B6DF18F09523FD
:104FB00009F0A2CFA7CF1124EACFC6DFA0F3959FB7
:104FC000D1F3950F50E0551F629FF001729FBB27F0
:104FD000F00DB11D639FAA27F00DB11DAA1F649F9C
:104FE0006627B00DA11D661F829F2227B00DA11D4F
:104FF000621F739FB00DA11D621F839FA00D611DD5
:10500000221F749F3327A00D611D231F849F600DF5
:10501000211D822F762F6A2F11249F5750408AF02E
:10502000E1F088234AF0EE0FFF1FBB1F661F771FBA
:10503000881F91505040A9F79E3F510570F05CCFFA
:10504000A6CF5F3FECF3983EDCF3869577956795A6
:10505000B795F795E7959F5FC1F7FE2B880F911DD8
:105060009695879597F90895DB018F939F930E94FA
:105070008E28BF91AF91A29F800D911DA39F900D8F
:10508000B29F900D11240895AA1BBB1B51E107C0CC
:10509000AA1FBB1FA617B70710F0A61BB70B881FC8
:1050A000991F5A95A9F780959095BC01CD01089557
:1050B00097FB072E16F4009407D077FD09D00E94C5
:1050C000442807FC05D03EF4909581959F4F0895A4
:1050D000709561957F4F0895A1E21A2EAA1BBB1B04
:1050E000FD010DC0AA1FBB1FEE1FFF1FA217B307B4
:1050F000E407F50720F0A21BB30BE40BF50B661FCA
:10510000771F881F991F1A9469F76095709580958D
:1051100090959B01AC01BD01CF0108950E94992893
:10512000A59F900DB49F900DA49F800D911D1124FB
:105130000895A29FB001B39FC001A39F700D811D70
:105140001124911DB29F700D811D1124911D089590
:10515000911106C080538A5010F0865C06C00895F5
:1051600099278827089585FDFBCF80629111F8CF9C
:1051700081568A51E0F708959111089581568A5118
:0C51800008F4805285580895F894FFCF81
:10518C000000220620005F01FE01DE01200020004D
:10519C00005301DE01DE0100000000003F3F3F0034
:1051AC003C4E554C4C3E00020057494445320001E0
:1051BC000057494445310041505A4D444D4E4F43E0
:1051CC00414C4C01010101013F3F3F003C4E554C0D
:1051DC004C3E00B103C803D003D103D503D20392D4
:1051EC00039803FF03A5039B03D2033031323334FE
:1051FC003536373839414243444546303132333401
:10520C003536373839616263646566252E3673002E
:10521C002D2564005741524E00455252003A252E1E
:10522C002A730A005352433A20005B252E36732D05
:10523C0025645D20004453543A2000504154483AB0
:10524C002000444154413A2000252E2A73000D0AB7
:0E525C000053657269616C20696E7075740094
:00000001FF
